:1000000000308A00F52A00000A108A100A118207BF
:10001000E134703471347234B034B134B234D03429
:10002000D134D234E034E23438308400000803198B
:1000300028280130F800F701F70B1C28F80B1B28C3
:100040004A30F700F70B222800000000800B192827
:10005000003483168613831286139630B80014205A
:1000600083168613831286179630B8001420003446
:10007000603083168F000F080439043C031D3B28B1
:1000800006138312061383168512831285168316B0
:1000900006108312061483168610831286148316A4
:1000A0000611831206150230B500C830B8001420BE
:1000B000B50B5528292029200230B500C830B800DA
:1000C0001420B50B5E28FF2ABA1B8E28BA08031D20
:1000D0006D283908003C03188E2883168611831278
:1000E00086110130BB003B083802031C7D2839080B
:1000F0000319BA03B903BB0A732883168611831246
:1001000086150130BB003B083802031C8D283908D6
:100110000319BA03B903BB0A832864280034031700
:100120008D018F0183168C130C1483120C0803139A
:10013000A000200F9D280130A000013003178D0082
:100140008F0183168C130C1483120C080313A10067
:10015000210FAC280230A100023003178D008F015F
:1001600083168C130C1483120C080313A200220FA5
:10017000BB280330A200033003178D008F018316C4
:100180008C130C1483120C080313A300230FCA282A
:100190000430A30000340C30B8004E30BA002030D8
:1001A000B90064200034831686138312861302304C
:1001B000B500C830B8001420B50BD92883168613B3
:1001C000831286170230B500C830B8001420B50B72
:1001D000E42800340230B500C830B8001420B50B54
:1001E000EC28831685148312B5018518B50A03100F
:1001F000350DB60083160514003083120518013042
:100200003604B500FF3A0339B500B508031D0D29C2
:1002100083160513831205132229350B142983161F
:1002200005138312051722293508023C031D1E29D8
:100230008316051383120513AC14222983160513A4
:1002400083120517CB200230B500C830B800142047
:10025000B50B2529AC1C3829AC100330B500C830CB
:10026000B8001420B50B2F29831605138312051728
:10027000D32000340230B500C830B8001420B50BCC
:100280003C29831685148312B5018518B50A03101D
:10029000350DB600831605140030831205180130A1
:1002A0003604B500FF3A0339B500B508031D5D29D2
:1002B00083160513831205177829350B64298316D5
:1002C00005138312051378293508023C031D6E2996
:1002D0008316051383120513AC14782983160513AE
:1002E00083120513AB01AA014230A9006830A800AF
:1002F000CB200230B500C830B8001420B50B7B29E4
:10030000AC1C8E29AC100330B500C830B8001420E6
:10031000B50B85298316051383120517D320D32027
:10032000DC2B0230B500C830B8001420B50B93297F
:100330005030B8007530BA003030B90064208316F0
:100340008613831286130630B500FA30B8001420E5
:10035000B50BA5298316861383128617DF2B02306F
:10036000B700C830B8001420B70BB1290B30B60065
:10037000B830B5003608FA0035080319B603B503DE
:10038000B7007A08B800B708031DC929B8080319CF
:10039000D82983168613831286134B30B800142095
:1003A00083168613831286177D30B8001420BA296D
:1003B000E52BB5013508023C031C712A3508FD3ECA
:1003C00003180B2A033E752A83160511831205159F
:1003D0008316851183128515831605128312051263
:1003E0000B2A8316051183120515831685118312B6
:1003F000851183160512831205160B2A8316051123
:100400008312051183168511831285158316051233
:10041000831205160B2A831606158312B7010619D7
:10042000B70A0310370DB800831686140030831204
:10043000861801303804B7000310370DB800831652
:10044000061400308312061801303804B700031078
:10045000370DB8008316851600308312851A0130D7
:100460003804B700370EF700F030F7057708F03999
:10047000B7003708F03C03196F2A00302C18013000
:10048000003A031D6C2A3230B80014202C14831655
:100490008613831286133230B8000130BA00F4306C
:1004A000B900642083168613831286173508B704B3
:1004B000B60136080B3C031C682A36080420F800F5
:1004C0003702031D662A3608F800742AB60A592A2C
:1004D000FF30F800742A6F2AFF30F800742AB50A3A
:1004E000DA292C10FF30F800E72B0A108A140A11C1
:1004F0008207E429F129FE2903178D018F010313D7
:10050000240803178C0083168C130C158312031315
:100510000B08F7008B138316031755308D00AA3094
:100520008D008C148C18922A0C11770883120313F7
:100530008B04013003178D008F0103132508031767
:100540008C0083168C130C15831203130B08F70011
:100550008B138316031755308D00AA308D008C1431
:100560008C18B02A0C117708831203138B04023005
:1005700003178D008F010313260803178C008316C1
:100580008C130C15831203130B08F7008B138316BF
:10059000031755308D00AA308D008C148C18CE2A8C
:1005A0000C117708831203138B04033003178D009B
:1005B0008F010313270803178C0083168C130C1567
:1005C000831203130B08F7008B13831603175530A0
:1005D0008D00AA308D008C148C18EC2A0C11770831
:1005E000831203138B048F20062C84011F30830594
:1005F000073083169F0086128312861638288316CA
:10060000851700308312851B0130003A031D942B9F
:100610000230B500C830B8001420B50B0A2B031700
:100620008D018F0101308C0083168C130C15831201
:1006300003130B08F7008B138316031755308D0037
:10064000AA308D008C148C18232B0C117708831280
:1006500003138B04013003178D008F0102308C00CF
:1006600083168C130C15831203130B08F7008B13DE
:100670008316031755308D00AA308D008C148C180A
:100680003F2B0C117708831203138B0402300317DE
:100690008D008F0103308C0083168C130C15831290
:1006A00003130B08F7008B138316031755308D00C7
:1006B000AA308D008C148C185B2B0C1177088312D8
:1006C00003138B04033003178D008F0104308C005B
:1006D00083168C130C15831203130B08F7008B136E
:1006E0008316031755308D00AA308D008C148C189A
:1006F000772B0C117708831203138B042830AD007D
:100700002D08093C03188D2B2D08B8000330BA00C2
:10071000E830B9006420AD03802B0230B500C8304A
:10072000B8001420B50B8F2B8F202008A4002108BF
:10073000A5002208A6002308A700AC10AE01AF0157
:10074000B301B201B101B001B41083168514831254
:10075000AD018518AD0A03102D0DB50083160514E3
:1007600000308312051801303504AD002D08FF3A22
:100770000339AD002D08023C0319BF2BEA203414C5
:10078000003034180130013C031DE62B2E08043CD8
:10079000031DE62BAE0120082402031DDE2B2108D9
:1007A0002502031DDE2B22082602031DDE2B230853
:1007B0002702031DDE2B3A293410E62B9129AF0ABC
:1007C0002F08023C0318E62BAF29AF01D92978087E
:1007D000AD002D0FEC2B192CB301B201B101B0010A
:1007E000B4102D080A3C031DF72BAE01192C2D085F
:1007F0000B3C031D0B2C003034180130003A031D54
:100800000B2C2E08043C031D062C7C2AEA203414F1
:10081000AE01AF01192C2D080B3C0319192C2E0821
:10082000033C031C192C2E08AE0A243E84002D081C
:100830008000003034180130013C031D682C013069
:10084000B0070318B10A0319B20A0319B30A00303A
:10085000B4180130003A031D482CB308031D3E2C88
:10086000B208031D3E2C3108413C0318482CFF3AC6
:10087000031D3E2C3008673C0318482CB301B2011D
:10088000B101B001B4148316861383128613682C49
:100890000030B4180130013C031D682CB308031D5F
:1008A0005F2CB208031D5F2C3108003C0318682C34
:1008B000FF3A031D5F2C30082B3C0318682CB30152
:1008C000B201B101B001B4108316861383128617EA
:1008D000A808031D742CA908031D742CAA08031D65
:1008E000742CAB080319912CFF30A807031CA9072F
:1008F000031CAA07031CAB07A808031D912CA90819
:10090000031D912CAA08031D912CAB08031D912CEB
:10091000EA203414AE01AF01B301B201B101B0015C
:06092000B410C02B6300BF
:02400E00103967
:00000001FF
